:020000040003F7
:10BC0000F03700200DBD030027BD030029BD030050
:10BC10000000000000000000000000000000000024
:10BC20000000000000000000000000002BBD030029
:10BC300000000000000000002DBD03002FBD030028
:10BC400031BD030031BD030031BD030031BD030030
:10BC500031BD03000000000031BD030031BD030011
:10BC600031BD030031BD030031BD030031BD030010
:10BC700031BD03004DBE030031BD030031BD0300E3
:10BC800031BD0300ADBE030031BD030031BD030073
:10BC9000CDBE030031BD0300D5BE030031BD03009E
:10BCA00031BD030031BD03000000000000000000B2
:10BCB0000000000000000000000000000000000084
:10BCC0000448854600F080F80048004761D1030031
:10BCD000C046C046F0370020056885F308884068F4
:10BCE000FF2464B2EFF30585002D01D1A64600477D
:10BCF0002546064621273FBAF0B400240025002639
:10BD00000027F0B4F92040B20047000003210948A1
:10BD100002680A430260084802680A430260074852
:10BD2000804707480047FEE7FEE7FEE7FEE7FEE73D
:10BD3000FEE700002405004054050040F5BE030066
:10BD4000C1BC030010B5202A04DB0146203A914013
:10BD5000002010BD914020239C1A0346E340194364
:10BD6000904010BD03460B439B0703D009E008C970
:10BD7000121F08C0042AFAD203E00B780370401C9B
:10BD8000491C521EF9D27047D2B201E00270401C29
:10BD9000491EFBD270470022F6E710B513460A464B
:10BDA00004461946FFF7F0FF204610BD30B50446A3
:10BDB0000020034600E05B1C934203D2E05CCD5CB4
:10BDC000401BF8D030BD0000064C0125064E05E0B2
:10BDD000E36807CC2B430C3C98471034B442F7D3AC
:10BDE000FFF772FF98F70300B8F703008307FF22FD
:10BDF000DB0E9A408907090E994000280BDA0007EC
:10BE0000000F0838830808489B001818C36993433B
:10BE10000B43C3617047830804489B001B181868D4
:10BE2000904308431860704700ED00E000E400E034
:10BE3000BFF34F8F04490348C860BFF34F8F00BF63
:10BE4000FDE700000400FA0500ED00E01CB5002449
:10BE50006846047000F06EFA03F0F2F9002818D179
:10BE60000E480168002914D00D498968C907C90F17
:10BE70000FD004600B4880686946087101A90A4820
:10BE800002F040F8084802F027F8002801D001F03D
:10BE9000B3FF6846007800F06BFA1CBD00D100408B
:10BEA00000D3004000D5004060F6030010B50649FD
:10BEB0000020086048608860C86003494039086015
:10BEC000486003F05BFA10BD4011014010B503F06B
:10BED000C7F910BD10B506484068002805D0804756
:10BEE000002801D000F0E0F810BD00F0FBFF10BD0D
:10BEF0006826002010B501F045F8002805D01F493C
:10BF00001D484860C8131E4988611E48018CC9B28B
:10BF100001290BD1828C120708D1028D1206120F53
:10BF2000042A03D1828D1206120F0AD0012921D1D1
:10BF3000818C09071ED1018D0906090F0A2904D039
:10BF400007E0114A01219160F5E7828D1206120F78
:10BF500005D00D290ED1808D0006000F0AD10B48A7
:10BF60000168012904D00A49016001680129FCD156
:10BF7000C021416110BD0000DFFF07C00005004087
:10BF8000006C0040C00F00F00006004000EC0640CE
:10BF90007593000030B47446641E2578641CAB426F
:10BFA00000D21D46635D5B00E31830BC184702E019
:10BFB00008C8121F08C1002AFAD170477047002034
:10BFC00001E001C1121F002AFBD17047202804DACA
:10BFD000012181400348014201D001207047002027
:10BFE00070470000FC06FFBC86B00B2269468A82BF
:10BFF00002220A7001234B7088700320C8700A71F6
:10C0000059204871FE20887102A805A901307DDF02
:10C01000002816D16846808A0B2807D8411C6A463A
:10C02000D17109210930117280B205E00C206946F6
:10C03000C871082008721420C1B200231A4668464D
:10C0400072DF06B07047000010B5144C86B0207A3D
:10C05000800702D5002006B010BD18216846FFF702
:10C060009AFE0620FFF7C0FF0028F4D16946087049
:10C070000190087228220A824882684673DF0028ED
:10C08000E9D1012006494005C860162001F0DCFE18
:10C09000A06802210843A060DCE700001026002011
:10C0A00000050050FFF7C4FEFFF7C2FEF7B5244CB1
:10C0B00082B060880E4681423FD800256846214FF5
:10C0C000057000F037F922786078A188884201DA9B
:10C0D000401C00E00020C0B2904204D168460078C5
:10C0E00000F046F927E065786078884201DA401C64
:10C0F00000E0002060706846007800F039F9BD4229
:10C1000019D0A068EF000499C151029900290CD000
:10C11000002E0AD0608832464543E0682818FFF7B1
:10C1200021FEA0683818868002E00021381881803E
:10C13000002005B0F0BD0420FBE70920F9E700006E
:10C1400028260020FFFF000010B50D4C03E0401C26
:10C1500000E0002020702078617881420FD02178A3
:10C160006088E26848438018A368CA00D1189A58CA
:10C17000898890472078A1888842EADAE7E710BDED
:10C180002826002030B5CB0008339DB29307002449
:10C19000002B01D0072030BD044B9A605219DA60A1
:10C1A0005C701C7058809980002030BD28260020CB
:10C1B0000A4B5B68002B07D0002A07D0002805D067
:10C1C0000068037C002B03D00820704707207047CD
:10C1D00000230374417442611846704748260020CA
:10C1E00010B50446082902D00020FFF75DFF216842
:10C1F0006068884710BD00001CB501910090034A9B
:10C2000008216846FFF752FF1CBD0000E1C1030092
:10C21000FFB507469007002581B01E46144600284A
:10C2200025D1002C23D002F077FD3046114EF0606E
:10C230003046103005704570029981704460756019
:10C24000357001240C487570240504600321142006
:10C25000FFF7CCFD09480460094CA76003211120B9
:10C26000FFF7C4FD6068B060002005B0F0BD072096
:10C27000FBE700003826002080E200E000E100E05B
:10C2800000150140FEB51F4B5B68002B30D0002825
:10C290002ED0052901D20720FEBD4369002B27D0EF
:10C2A000437C012B26D000270291044600256946D5
:10C2B00016460D70684600F03DF801A803F0DAF864
:10C2C000002819D0012101700F494460496881603C
:10C2D000029907614661C16068460A490079487061
:10C2E0006846007800F044F802F0FCFF2846FEBDE6
:10C2F0000820FEBD0F46D7E768460425007800F009
:10C3000037F8F3E7482600200015014010B508492A
:10C31000496800290AD0002808D04169002905D0C1
:10C3200000210174022103F005F810BD082010BDA2
:10C330004826002030B5EFF3108172B6094A5468E0
:10C340000123002C04D00370002900D162B630BD57
:10C350005360054B1D68054C254015601C6000228C
:10C360000270F1E75C26002080E100E0FC06FFBCE3
:10C3700008494A68002A0CD000280AD1EFF310803F
:10C3800072B60A68044B1A6000224A60002800D185
:10C3900062B670475C26002000E100E070B50546FB
:10C3A00001461C220E48FFF7DDFC0E4C00262670CD
:10C3B0002968002906D00822201DFFF7D3FC201D84
:10C3C0007ADF02E00748001D7BDF002807D1401E0E
:10C3D00060806670044A00210448FFF7E9FE70BDE2
:10C3E0000C2C0020FC25002011F40300F4F50300C0
:10C3F000F8B5214C0146028800261E48E589102A1E
:10C4000013D01E4F112A1FD0122A2BD0502A1AD116
:10C41000881DC988A94216D14189022913D10C303F
:10C4200000F016F900280CD112E08A8804464280F8
:10C43000104808220C301831FFF794FC6670002D6C
:10C4400001D100F0B5F9F8BD0021C9434180467023
:10C450003868FFF75BFF0028F5D0A1690029F2D00A
:10C460008847F8BD034808220C300831FFF77AFCF2
:10C47000E7E70000FC2500200C2C0020F4F5030069
:10C4800010B502480068FFF741FF10BDF4F5030046
:10C4900070B505460020C043134C86B020800126AD
:10C4A00068468674114901822A4604A93046A0DFF5
:10C4B000002817D10E4B0FCB03936B4607C3A91C63
:10C4C000684663DF00280DD1284600F09DFB002858
:10C4D00008D1284600F096FA002803D1A06830431E
:10C4E000A060002006B070BD1026002059FE00009C
:10C4F000FCF5030070B51A4D0024A868410701D56A
:10C50000002070BD04210843174AA8601549174B45
:10C51000126800BF00BF00BF00BF00BF00BF00BF68
:10C5200000BF9A4200D000BF0139F2D12A881049D9
:10C530008A4205D01321104676DF0400E1D10BE0DA
:10C54000800709D574DF0400DBD1152001F07CFCE5
:10C55000A86802210843A860FFF792FF204670BD3B
:10C5600010260020C0D401007C2600200024F40006
:10C57000FFFF000000B587B0152001F05BFC16201E
:10C5800001F058FC152001F05FFC162001F05CFC66
:10C5900024480068059001F085FA002817D1224848
:10C5A00013DF002813D1214B4822214905A802F0AE
:10C5B0001BFE002801D0FFF777FD01216A460846DF
:10C5C00002F0E6FD002802D1684602F0D7FD0028FF
:10C5D00026D1184802F0C8FD002821D100F052FCF5
:10C5E00000281DD112484830FFF752FF002817D10C
:10C5F0001C216846FFF7CFFB0F4801900120800304
:10C6000002900320694608730020C88108740B4813
:10C6100006906846FFF7C2FE002801D1FFF714FD1F
:10C6200007B000BDF8F5030000BC0300CDF1030026
:10C63000282C002041C60300CD0C0000A9C7030030
:10C6400010B50446FFF7D4FE204601F0B3FC10BD40
:10C650004178027808021043C007C00F70470000FD
:10C6600010B50349085C012101F0F6FB10BD000084
:10C67000ECF5030010B50349085C002101F0ECFB68
:10C6800010BD0000ECF503007CB50024074E2546E4
:10C69000305D0122009500231146019501F0B6FBA3
:10C6A000641C042CF4D300F003F87CBDECF503000B
:10C6B00010B500242046FFF7D3FF641C042CF9D3E7
:10C6C00010BD10B543689C184460002904D105E0F2
:10C6D00018780870491C5B1C521EF9D2012010BD4D
:10C6E000002807D00449814204D80449814201D975
:10C6F00001207047002070478026002090260020EF
:10C70000F8B52348416800293ED00E6821494C689D
:10C7100087688078E11B0D022D0AED1C002814D1DA
:10C7200001201D4A000450601B4A403A50601B49DA
:10C73000400008601A4908601A49012008602F204B
:10C7400000F066FD124901208870B54200D23546DE
:10C75000E81900020F4B000A403318600D4A516877
:10C76000001B091B0902090A0002000AC91C8142B8
:10C7700009D9506818602F2000F04AFD01200749B0
:10C78000400480390860F8BD02F0C6FAF8BD000028
:10C7900038260020001501404013014080E200E0EF
:10C7A00000E100E00010014010B5FFF77DFC10BD76
:10C7B000F8B5164800F0D8FB144D00260C3D144C7B
:10C7C000002807D0616900291CD001206A4610703A
:10C7D000684616E02878002805D06169002911D044
:10C7E000684606700DE0687800280DD0A1680948F9
:10C7F00000220068FFF746FD002803D0A169002948
:10C8000000D088472E70F8BD6168F0E70826002048
:10C810000C2C0020F4F50300F0B50026F643002AA6
:10C8200004D01268D2430023094F0DE03246FAE7E4
:10C83000C45C624008245508D20700D032463A4012
:10C840006A40641EF7D15B1C8B42F1D3D043F0BD2C
:10C850002083B8EDF0B5146907462068251D8DB01A
:10C860001646002819D002291BD00A2000906B46DA
:10C8700009AA384602F0ABF900280CD009A901A892
:10C88000009A02F081F801AF0FCF0FC723687168DB
:10C890002A4605A898470DB0F0BD384602F0E8F8E2
:10C8A000F9E76946384602F077F80028F3D02368A4
:10C8B00071682A46684698470028ECD002980028FC
:10C8C000F5D1019878600120E5E710B553685B78F1
:10C8D0009B099B0103D0402B04D0002010BD00F029
:10C8E00005F810BDFFF7B6FF10BD0000F0B50F460C
:10C8F00051680646487814460207120F324D9300DD
:10C90000ED58302385B0184006D0102806D02028D6
:10C9100008D0302855D140E022694FE061690120FC
:10C92000087049E0022F2AD1042A28D8012000905B
:10C9300001A93046676902F02FF800281DD00AE0EF
:10C940000A7942432069121801A8A847002810D08C
:10C950003878401C38700398002804D06168387813
:10C960004A799042ECD3029870600398002828D14D
:10C9700002E000200090F6E7009805B0F0BD626983
:10C980000B791078276943434979DB19884218D21B
:10C99000401C10701A46616810E008786169072A27
:10C9A000087009D1606801792069FFF7F4F96068BF
:10C9B0002169806802F00BF8226961683046A84757
:10C9C000DBE70020D9E7000074F7030010B50B493E
:10C9D00009480B4A096800BF00BF00BF00BF00BF85
:10C9E00000BF00BF00BF914200D000BF0138F2D1AC
:10C9F000FFF7AAFB10BD0000A08601007C260020E6
:10CA00000024F40030B58FB004461C216846FFF7BF
:10CA1000C2F9142109A8FFF7BEF900206946079062
:10CA20000A7808210A4310231A4369460A70A2783B
:10CA300008A98A700125694602070D84120F0A773A
:10CA4000EA184A778A7FF9210A40921C1A432A433E
:10CA500069468A7708A9099107A917220A916946A8
:10CA60000A860D90234620880C3309AAA2DF0FB056
:10CA700030BD000002488168491E81607047000097
:10CA8000E02500201FB50E480146826B5C316846E8
:10CA900001F07AFF6C460ECC0A480EC009490A48DC
:10CAA000C8600A49002008604860094A09490548E9
:10CAB00001F002FD002800D0012004B010BD0000EC
:10CAC000B82F0020DC2B0020F9E70300F42500201C
:10CAD00090260020C8F5030070B50024001D002A30
:10CAE0002BD0002B29D05F21095C002903D06021C5
:10CAF000095C012921D0017A00291ED0C16833299F
:10CB00001BD1002103231B03027C14E08D002D1890
:10CB10009E896D69B6B2B5420CD1014620314B7980
:10CB2000354A002B0BD0012B12D0022B0CD0032B3B
:10CB300003D109E0491C8A42E8DC0A2070BD047870
:10CB4000002CFAD0946803E00478002CF5D0D46867
:10CB5000002B04D0022B06D0032B07D103E0426840
:10CB6000A242EAD302E04268A242E6D90022234C64
:10CB7000002B22612BD0012B34D0214AFF25AD029E
:10CB8000AA1A022B28D0032BD7D10B7B002BD4D091
:10CB900089790029D1D0836A016B5D182561002B4A
:10CBA00026D0002924D091420FD8014620223F31BF
:10CBB0001448FFF7D7F82069002819D00F4A002140
:10CBC0000C3200F001FE002814D0042070BD097D55
:10CBD0000029B2D0816B09E0097B0029ADD0016B3F
:10CBE0002161E0E789790029A7D0816A2161DCE72A
:10CBF000032070BD012070BDB82F0020E02500206B
:10CC000000BC0300BC2B002010B58EB004461C21D4
:10CC10006846FFF7C0F8142109A8FFF7BCF8002206
:10CC20006946079208780421084369460870A0788D
:10CC300008A98870022069460884501C0007000F6C
:10CC40000A7710304877887FF92108400121801C3D
:10CC500008436946887708A8099007A80A90142015
:10CC600008860D922088231D09AAA2DF0EB010BDF0
:10CC7000044A002901D1002313705268002A00D011
:10CC8000104770472026002010B50E4900230A786F
:10CC90004C78A24212D0521CD2B20A70022A00D1A1
:10CCA0000B700A78074B920018339A580260886814
:10CCB00010180002000A8860012010BD03600020E7
:10CCC00010BD000038260020F8B506461C481F4657
:10CCD000007815460C46C0070AD03046FFF700FD25
:10CCE000002807D0002C07D0A00507D00620F8BDEB
:10CCF0000120F8BD0220F8BD0320F8BD3068A04235
:10CD000004D8A80271680019884201D90520F8BD2D
:10CD1000002D10D0684601F0EFFE00280DD00098DD
:10CD20000221C0C00170A101090C8180058101F0C0
:10CD300035FF0020F8BD0420F8BD0720F8BD000035
:10CD40006426002030B4094B02241A6852085200AD
:10CD50001A60002906D022431A604268002A03D0D4
:10CD600030BC1047A243F7E730BC70471C260020B8
:10CD70000348012201781143017000207047000030
:10CD8000642600200348406E042801D0002070472C
:10CD90000120704744310020F8B507461E481E4662
:10CDA000007815460C46C0070ED03846FFF798FCB1
:10CDB00000280BD0002D0BD0002C09D02846204392
:10CDC000800707D00620F8BD0120F8BD0220F8BD7D
:10CDD0000320F8BD3868A04204D8B100786809196A
:10CDE000884201D20520F8BD002E11D0684601F01E
:10CDF00083FE00280ED0009806990760416001214B
:10CE00000172C5600461868201F0C8FE0020F8BD91
:10CE10000420F8BD0720F8BD6426002070B5174B2C
:10CE20000446186E182148431549C0180A7895071A
:10CE300015D5022C02D0032C1CD102E001F0B4F96C
:10CE400018E04A78521CD2B24A70032A12D9002242
:10CE50004A70082101F0C4FF01F038FE0AE05007D3
:10CE600008D5FB2002400A70586E002802D002202C
:10CE700002430A7001F05CFE70BD000044310020E6
:10CE80006426002010B5002486B0601C0007000F47
:10CE90000194694610300294087003A871DF0028DD
:10CEA00019D16946487B401C487303A9002070DFF4
:10CEB000002810D1072209A168467CDF00280AD18A
:10CEC0000C21684681801821C180FF2104819131A5
:10CED000418101A87ADF06B010BD00004466755498
:10CEE00061726700F8B51F4C2078002839D020699E
:10CEF000002807D00026E068002805D00025002E75
:10CF000004D014E00126F6E70125F8E76078002850
:10CF100027D1684652DF052804D0002804D0FFF747
:10CF2000C3F804E0012602E0216900988847002D3B
:10CF300013D16078002814D1608869460880A06801
:10CF400061DF052804D0002804D0FFF7ADF804E025
:10CF5000012502E0E168A0688847002ED6D0002DA8
:10CF6000CDD0F8BD6826002041880548028891424E
:10CF700004D34088814201D80120704700207047C7
:10CF8000002600201048018CC9B2012917D1818CDC
:10CF9000090714D1018D09060A0F03D1828D1206EB
:10CFA000120F0ED0090F012903D1828D1206120F24
:10CFB00007D0032903D1808D0006000F01D0002087
:10CFC0007047012070470000C00F00F070B50546A3
:10CFD00008680C4686684A683146284601F01EFCFF
:10CFE0006068286120460C306861707880090228EA
:10CFF00001D1241D2C6170BDF0B5284C214610399B
:10D0000048688B68227886469C46CF78667836E0FA
:10D01000182353436168521CC918A378D2B29342B3
:10D0200000D100220B78022B02D0032B27D123E062
:10D0300003464D68194603E0A94204D00B46C9696E
:10D0400000291CD0F8E7002919D08B4208D1C0690B
:10D05000002805D1124F0125BD600025AC460127EF
:10D060000D68C969D961002909D00B685B190B608B
:10D0700005E00174C06900E000210028F9D1964262
:10D08000C6D10649624610398A604860CF70704543
:10D0900001D00120F0BD0020F0BD00004826002096
:10D0A00000100140F8B52C4E044670680025009031
:10D0B00041E0002C02D02046E46920E026481823F5
:10D0C0001030017842684B43491CC9B2D218017034
:10D0D0008378994200D105701178506801292CD1CC
:10D0E000017C002929D191684160D1688160116972
:10D0F000C16051698161F178002900D045604368C1
:10D10000B268164F991A0902090AB94202D2826816
:10D11000891806E0D11A09028268090A8A4202D9EE
:10D12000511A016000E005604560012185600174CD
:10D13000C56102F0DFF8002CBBD107481030017840
:10D1400040788142BAD171680098814201D00120B3
:10D15000F8BD0020F8BD000038260020FFFF7F004A
:10D1600010B5FFF791FA0220FFF784FA0849074843
:10D17000086000F023F8002801D0FEF759FE0320D4
:10D180000003806800F006F8002010BD0C000300CA
:10D190005007005010B5044600F084FC002809D167
:10D1A0000549401E0860204613DF002802D12046B2
:10D1B000FEF792FD10BD000080E100E010B500F028
:10D1C000D7FB10BD70B59CB01C4615460E46052811
:10D1D00002D006201CB070BD6068202801D0092054
:10D1E000F8E7684601F0BCFE0028F3D12A46314634
:10D1F000684601F091FF0028ECD1012268462168C1
:10D2000001F026FE0028E5D1202060600020E1E743
:10D2100000280FD00849094A096800BF00BF00BFB5
:10D2200000BF00BF00BF00BF00BF914200D000BFE1
:10D230000138F2D1704700007C2600200024F40061
:10D24000F1B50320274D00038268286B6E6A12181F
:10D2500082B0371A00920124A402A74200D83C46AB
:10D2600000220121009800F0E9FA002838D10023BB
:10D2700022460299009800F043FB002830D1224654
:10D280000299009800F0E2FB002829D10022012138
:10D29000029800F0D3FA002822D1286B00192863E5
:10D2A000002000F03FFD009800190090029800193E
:10D2B00002903F1BCFD1032000038068002231463B
:10D2C000FFF7AAFAA96A814203D10121AE6129625E
:10D2D000E8610448243000F0ADFB002000F022FD9E
:10D2E000FEBD0000B82F002010B50A4C206A0128AE
:10D2F0000CD1E06900280BD003200003A1698068ED
:10D300000022FFF789FAE169814201D0002010BDB7
:10D31000012010BDB82F002070B50D460A680B49DA
:10D32000496B541A0E1822463146094800F08EFB0C
:10D33000002804D02146304600F096FB70BD2846F8
:10D3400000F078FB002000F0EDFC70BDB82F00204D
:10D3500000BC0300F8B51446404F0A780E4601257C
:10D36000B96BF86B1300FEF715FE077605203B1C22
:10D37000766E7600B068002805D0FF210131884222
:10D3800003D90420F8BD0320F8BD3548002484707B
:10D39000324820213830FEF7FEFC3C63B068B863A9
:10D3A0005AE06060386CA06056E0B26813188B4297
:10D3B00003D96060386CA060E5E7284B71685C3386
:10D3C000C018FEF7CFFCF86BB168244A4018F86328
:10D3D0004032B1687068FFF71FFA3864F86BE0E715
:10D3E000884201D00820F8BD1D4CA078002801D04B
:10D3F0000120F8BDFFF746FB012822D11948007D26
:10D400000028194818D0783082781849012A01D0AC
:10D4100005200CE0124A14320CCAFFF75DFB01280C
:10D4200005D1002000F07EFC002802D00A2005462D
:10D4300012E00120A0700FE00078002801D00A253A
:10D440000AE00520F8BD386CA060F86B6060FF2032
:10D450000130206000E002252846F8BDB82F0020EA
:10D46000E0250020F026002090260020DC2B002064
:10D4700010B5024603200A4B0003816818461C6958
:10D480001830012C08D05C69002C05D09B69054C34
:10D490000C301B19A343591800F006F810BD00000A
:10D4A000B82F0020FF030000F8B50D4616460146D0
:10D4B0008A680020012A0DD00127A52A12D0AA2AA5
:10D4C0001ED0AC2A0DD10C46284600F0BFFB002828
:10D4D00014D119E00F494969012902D12846FFF703
:10D4E000AFFEF8BD28460C4600F0B0FB002805D181
:10D4F000204600F09FFA002000F014FC3760F8BDD1
:10D500002846FFF709FFF8BD21462846FFF704FF2C
:10D51000F4E70000B82F0020FEB5012000909748E6
:10D520000E788078964F019015460C46BA6C396D8E
:10D53000786D3300FEF72EFD07F2053AF7F3F2EFB0
:10D54000F200A168002946D08C4A8B05126902D0EE
:10D55000431893423FD101231B03994232D8019BC8
:10D56000864D002B7ED0411891427BD8F96CB9646E
:10D57000A1683865796438636978824A491C8907EB
:10D58000890F69700021A980A968491CA960A16858
:10D590008918EA68890A80187B4A00F04FF9002848
:10D5A0007ED0A868401EA8600520FEBD6960B86CEA
:10D5B000A8600198714E0028D4D0FF20A1680130E6
:10D5C000814201D90420FEBD386D7A6D0818801A99
:10D5D0007A6C904201D90320FEBD694A60684832E6
:10D5E000FFF71AF966498864086DA2688018086513
:10D5F0006860886CA860B088A2681118FF2907D8F5
:10D60000717867680B02614959180818394643E078
:10D61000FF210131091A8FB2717863680A025B49F0
:10D62000511808183A461946FEF79CFBB088C019F5
:10D6300082B2B280A068D21CC01BA0606068920851
:10D64000C0194F4F6060386BF1684018B168491CD1
:10D65000B16071780B024D4959184B4B00F050F9ED
:10D66000002800E063E04CD0B068401EB060F86C69
:10D67000B864786D38656860F86CA86070780021CF
:10D68000401C8007800F7070B180A268002A71D0A2
:10D6900003023E4861681818FEF764FB208900E029
:10D6A0002EE0B18840180104B080090C62D0344CDF
:10D6B000626D206B636C821A52189A425AD3F268D8
:10D6C000C91C8018B268521CB2608A0871780B02BB
:10D6D0002E4959182C4B00F013F9002816D0B068C9
:10D6E000401EB060E06CA064606D20656860E06C16
:10D6F000A8607078401C8007800F70700020B08098
:10D7000038E0B188386B40183863B7E7B188206BD0
:10D7100040182063EDE727E001E004E02CE06960B9
:10D72000B86CA86026E07B6C081A984201D00820EB
:10D73000FEBDFA6400207965786400F0F3FA0028F1
:10D7400001D00A20FEBD0D4C386D2169884202D0FF
:10D7500010E000F04DFBA0680028FAD10B48B0386B
:10D7600000F0ACF9009005E0AA60386D6860012017
:10D77000000328600098FEBD0220F3E7E0250020AA
:10D78000B82F0020FF03000075CA0300BC2700204B
:10D7900010B50B480069000DC007C00F0ED0094836
:10D7A000816D012901D0002010BD0021816508464E
:10D7B00000F0B8FA002801D0FEF776FC012010BD79
:10D7C00000050050B82F0020F0B58C4618490324FE
:10D7D0004B69032109038968A4025B1A1F1B874256
:10D7E00015D3144C11602346183B196A00250129F2
:10D7F00001D01D610EE0104E216889198E0AB60213
:10D80000BF1B0121B84207D96246002A01D004207B
:10D81000F0BD19615D6106E01D61064C596111683A
:10D820000C34711811606560A56020600020F0BDA7
:10D8300000100010D02F0020FF030000F0B50E46AE
:10D840002049044608681546002785B0420719D5C7
:10D85000820702D50A2005B0F0BD01221949104304
:10D860000860B2B22B4621461748FFF72DFA070091
:10D870001448016802D04908490001E0012211431F
:10D8800001601DE0A001000C0490204600F0F0FAB9
:10D89000012080022418761EF7D1002D10D00B4AEB
:10D8A00091681068D26802910090019503926946D0
:10D8B00004980881A001000C488100216846A8470F
:10D8C0003846C8E71C260020802600200CF60300FE
:10D8D00010B501460020084C00290BD0FFF748FA8C
:10D8E000002804D1054801F0B1FC002801D008202F
:10D8F00010BD0421216010BD1C2600201DCE030098
:10D90000F0B51646184A074610681C46002585B033
:10D91000430717D5830702D50A2005B0F0BD0123C0
:10D92000114A184310600A46B3B239460F480094B2
:10D93000FFF732FA0500F0D10B48012201681143CC
:10D9400001600EE03246384600F0A8FA002C08D0FC
:10D950000020009003900297019468468681002180
:10D96000A0472846D9E700001C260020802600207A
:10D97000F8B50020009000F0ADF96846FFF778FD9B
:10D980000125002800D00095FFF702FF002801D0F4
:10D99000009511E0009800280ED1FFF7A5FC0028A3
:10D9A0000AD0FFF7A1FC002804D003200003806800
:10D9B000FFF7F0FB0020F8BD184B194A05210020A5
:10D9C000FEF726FC002801D0FEF76EFB144A142156
:10D9D00078320820FEF7D6FB002801D0FEF764FB62
:10D9E00000F0F0F90028E6D100F0E4F80D4F0E4CFD
:10D9F0000E4D0F4E386800280DD001210020A3687D
:10DA00000A468240134202D0820092191560401CDF
:10DA1000C0B20728F3D3FEF797FBEBE7F9C1030089
:10DA2000942C002000040140000501403546526E50
:10DA300000060140002101604160816002480163ED
:10DA40004163016141617047B82F00201FB5054B4C
:10DA500092081B6A01AC009307C4684618DF04B043
:10DA600010BD00001CF603001FB58908002201ABA1
:10DA7000009207C3684618DF04B010BD1FB59208B6
:10DA800013061B0E02D0092004B010BD044B1B6806
:10DA90000290009303920191684618DFF4E70000BA
:10DAA0001CF603001FB5044B6C460FCB0FC4684631
:10DAB00018DF04B010BD00002CF60300F8B50746CF
:10DAC00004462037787F0125032808D00A25354EE3
:10DAD000706900281DD001281ED00A20F8BD334EE1
:10DAE000314830602020334670601846143802698F
:10DAF000C1680520FFF766FB002800D00A252146F3
:10DB000020223F313068FEF751F90028DFD005258B
:10DB1000DDE72448183001E022482430012D03D0ED
:10DB200000218160416027E0797900290ED0012928
:10DB30000ED002290ED003290FD00A2579790029A9
:10DB400010D0022911D0032911D10EE0012102E0E9
:10DB5000A52103E0AA218160F0E7AC218160A16AE0
:10DB60007163EBE76168B16001E06168F160B16C1D
:10DB700041600E491439096901600A482021383092
:10DB8000FEF709F90748FF22B2215C30FEF7FCF8E6
:10DB900000203063064800F0C5F8002800D00A25B0
:10DBA0002846F8BDB82F0020BC2B0020F42500200B
:10DBB00089E1030070B50120FFF78AFE002821D11A
:10DBC000114D124CA860A06B00281AD0FEF75AFF26
:10DBD000002816D0206A00280BD1A069002808D0A0
:10DBE000094A00210C322861FFF7EEFD0120A870E0
:10DBF00007E0E06A002804D1A069002801D0606A2B
:10DC0000EEE7002070BD0000E0250020B82F0020C6
:10DC100010B50C780C4B012C01D0062C07D10C79D7
:10DC2000012C03D0022C01D0072010BD1C701B78E2
:10DC3000012B03D0022B04D0052010BDFFF78AFB77
:10DC400010BDFFF769FC10BDE0250020F8B50346C4
:10DC500019480122016B12038E18426B174D541A9A
:10DC60006419AC43A7087D19AD0AAD02CF18002A8C
:10DC700003D0914201D10020F8BD2A4639463046F2
:10DC8000FFF7FCFE0028F7D12A4639463046FFF759
:10DC9000DDFE0028F0D176197F19A54201D90024B4
:10DCA00000E0641B0448416B091B0163002000F085
:10DCB00039F8002CE1D1F8BDB82F0020FF03000097
:10DCC00010B5002258210248FEF7A6FD10BD000045
:10DCD000BC2F002070B5104900200870FF255D356D
:10DCE0002A460E490E48FEF73DF80D4C2068401CB0
:10DCF00004D0FFF7E5FF216881420CD0294608488F
:10DD0000FEF749F801206060002000F00BF80028C1
:10DD100001D0FEF7C9F970BD2026002000FC0300E9
:10DD2000B82F002070B50546164C01E0FEF74EFEF8
:10DD300020780028FAD101202070656001F0B0FB46
:10DD4000002201211048FFF779FD0728F6D00025B1
:10DD5000002814D1FFF7B4FF0C49FF225D320860A0
:10DD6000881AFDF7FFFF01F09BFB094B5722094979
:10DD70000548FFF7C5FD0728F5D0002801D025701C
:10DD8000032070BD2026002000FC0300B82F0020D7
:10DD900071CC03005C2E002070B50848084D401B74
:10DDA000C6080020044606E0E000401940688047AD
:10DDB000002802D1641CB442F6D370BDC0F7030042
:10DDC000B8F7030070B50848084D401BC60800208E
:10DDD000044606E0E000401900688047002802D1B0
:10DDE000641CB442F6D370BDC0F70300B8F703005B
:10DDF00010B5FEF7A9F910BD02490120886002495B
:10DE00000860704700D3004004D0004070B5520055
:10DE10000A439900049D0A432902059E0A433104DE
:10DE200005240A432407800007210019090240182D
:10DE3000026070BD052212078000801807220321AE
:10DE40001202801801607047012181400148816001
:10DE5000704700000005005001228240034800295D
:10DE600001D082607047C26070470000000500501A
:10DE7000084A0221516008490B68002BFCD09060D1
:10DE800008680028FCD00020506008680028FCD0FA
:10DE90007047000000E5014000E40140F0B50C4D82
:10DEA00001236B600B4C2368002BFCD0002306E0A1
:10DEB0009E008F5987512668002EFCD05B1C934230
:10DEC000F6D30020686020680028FCD0F0BD000078
:10DED00000E5014000E40140016880684A68824230
:10DEE00001D2521C00E000220868824201D10120C8
:10DEF0007047002070478068884201D9481C7047ED
:10DF000000207047FEB504460E4600206946019089
:10DF100008706846FEF70EFA2046FFF7DDFF07009F
:10DF20000AD0207C002807D00420019068460078A1
:10DF3000FEF71EFA0198FEBD2068416820460D4696
:10DF4000FFF7D9FF2168002F486006D020680168DC
:10DF50002046FFF7D0FF21680860E268012A15D04B
:10DF6000022A17D0042A1AD0082A1DD01046616848
:10DF7000684308183146FDF7F5FE204600F01CFE08
:10DF800021688A688242D1D28860CFE761683078A0
:10DF90004855F2E7616830886A008852EDE76168A9
:10DFA0003068AA008850E8E7626803CEEB00D21818
:10DFB00003C2E2E770B50446314D00882E8814286C
:10DFC0004CD00DDC022836D010281CD0112828D0C7
:10DFD000132817D100231A46852130467FDF0DE034
:10DFE000502847D051282AD052283DD0552809D151
:10DFF000A079002806D11321304676DF002801D011
:10E00000FEF752F870BD01201E498005C86015203A
:10E01000FFF71AFFA0882880A86802218843A8601B
:10E0200070BDFEF711F8002801D0FEF73DF8002082
:10E03000C043288070BD0021304667DFDEE7A0794D
:10E040000028F7D02146104800F0D8F80028F1D079
:10E05000214608310C4800F019F870BD0023A08853
:10E060001A46194686DFC9E70023A0881A461946D2
:10E07000A9DFC3E72146044800F008F970BD00009D
:10E080001026002000050050702C002030B50446FA
:10E0900087B00020059003900490009001900290BA
:10E0A0000D7B38482B00FDF775FF076A052D3B23D4
:10E0B0006A4E6A004A89062A01D0032216E0428885
:10E0C0008280487B0190087C4A7C00041206104341
:10E0D000CA7B8B7B110219430843029001206946D9
:10E0E000087003AA0020FFF793FD024601213CE0DF
:10E0F00003206946087003AA0020FFF789FD024645
:10E10000042132E04A89032A01D0032206E08A7BF7
:10E110004B7B11021943418081800122022124E0BE
:10E1200004206946087003AA0020FFF771FD02462B
:10E13000012801D0032118E02046059A049900F037
:10E1400075FD07B030BD4889022801D003220BE0DD
:10E15000487B019006206946087003AA0020FFF75B
:10E1600057FD0246012804D00621204600F0B8FDE4
:10E17000E7E703AD0ECD204600F082FDE1E7032284
:10E180002946F2E710260020FFF706FEBFF34F8F67
:10E1900004490348C860BFF34F8F00BFFDE700008C
:10E1A0000400FA0500ED00E010B5134A002151709B
:10E1B000017A012911D002290ED18189491C81815E
:10E1C000C189491C89B2C181028A914204D10021CE
:10E1D00000F006FE00F07AFC10BD838AC28A991A0C
:10E1E000FF2901DC89B201E0FF210131511889B218
:10E1F000C1829942EBD010BD6426002030B587B0B3
:10E20000002401940294039404948A1D8B790831AC
:10E21000022B33D153888589AB422FD1127A042A3D
:10E220002CD0062A2AD0052A28D002236A46137148
:10E23000012595720D8995814D89D5810C31059403
:10E24000049193820692104D018A05AA2888A5DFC1
:10E25000002804D16846FEF7FBF9002807D068467D
:10E26000048101A92888A8DF00280AD006E0FF2041
:10E27000FE306946088101A92888A8DF002007B080
:10E2800030BD0120FBE700001026002030B5054618
:10E29000C888AA8887B0904223D1002005900390B7
:10E2A00004900090029002206A46107008461230D6
:10E2B0000190088A029003AA69460020FFF7A8FC93
:10E2C000094C608800280CD0A088401E0004000C77
:10E2D000A08006D12846059A049900F0A7FC608822
:10E2E000A08007B030BD000010260020F8B50D4614
:10E2F00014460646694600F058FA00280DD0009BE7
:10E30000FF2B09D8581C834206D86978890902294D
:10E3100002D02979814201D20020F8BD2370611C0E
:10E320003046009A00F066FBF8BD10B5114600F0CB
:10E33000D1F810BD10B5114600F0E1F810BDF8B5E8
:10E340000C4615460646694600F02FFA00280BD009
:10E35000009A501C904206D361788909022902D0A4
:10E360002179814201D20020F8BD2946304600F0D3
:10E3700041FB009A0021A954F8BDF0B585B00C46C8
:10E380008E6817460546694600F006FB00280ED049
:10E39000A06800280BD060783A468006800F0228DB
:10E3A0003146684605D000F0D7F80199696005B09C
:10E3B000F0BD00F081F8F8E77CB50D4614466946DB
:10E3C00000F092F900281FD02879082806D00428E8
:10E3D00008D0022809D001280BD014E00098019938
:10E3E00003C40AE00098206006E0009800B2208094
:10E3F00002E0009840B22070C117009A019B504083
:10E400005940084301D000207CBD01207CBD7CB573
:10E410000D461446694600F0A5F900281FD028795A
:10E42000082807D00021042808D0022809D0012894
:10E430000BD013E00098019903C409E00098206014
:10E4400006E0009880B2208002E00098C0B2207000
:10E45000009A019B50405940084301D000207CBDE8
:10E4600001207CBD7CB50D461446694600F07AF962
:10E4700000281ED028790099082807D0CA17042838
:10E4800009D002280AD001280BD011E0019A06C455
:10E490000846134608E00846216004E008B22080E0
:10E4A00001E048B22070C31748405340184301D0E0
:10E4B00000207CBD01207CBD70B50D46064614468B
:10E4C0001146284600F083FA22462946304600F0DD
:10E4D00043F870BD38B50C460422694600F08AFA4C
:10E4E00000280BD06846807801046846C078000692
:10E4F00001436846008801430120216038BD1CB5F6
:10E500000C460822694600F075FA002823D06946B7
:10E510000A784978080E09020A4369468B78190C73
:10E520001B0408431A436946CB78190A0843694615
:10E5300009791B060843694649791A4309020843C9
:10E5400069468979090408436946C9792260090640
:10E550000843606001201CBDF0B5054600209DB059
:10E5600001900646029004A800F058F98BE003AB36
:10E570000AAA6946284600F0D2F800280BD004A861
:10E580000A9900F05CF900280BD0059840788006C5
:10E59000800F59D066E06846007B002878D11DB016
:10E5A000F0BD0A98B04249D3059C04AE0598407866
:10E5B0000007000F082814D0304600F057F90598DE
:10E5C000A042F3D10026F6430A98B04236D3A96898
:10E5D00011910C90684600780B9008980468169189
:10E5E00022E005980678EFE720680768002F05D03D
:10E5F000214628460B9B0C9AB84712E012952068DA
:10E600000C9980680B9F007888420CD1214617A88E
:10E61000FEF7DCFC0121217317AA39461298FEF798
:10E6200054F90028BBD0A468002C03D0A968169820
:10E630008142D9D0A9681198814224D168460178D5
:10E64000284600F015FA1CE0069840280AD2C006B9
:10E65000C00E0121814006984009820001A883581C
:10E660000B438350EC68002C05D06846027804AB5D
:10E6700028460A99A0476846017804AA2846FEF76A
:10E6800024F900288BD0A868002801D06FE7FFE7A5
:10E690000598069C457804A800F0E8F80028F7D112
:10E6A000A806800F04D105980078002800D0641CCB
:10E6B000002C17D0002001A9630904E082008A58C9
:10E6C000521C0DD1401C8342F8D898000A58E0062D
:10E6D000C00E2021091A0020C043C840824201D048
:10E6E00000205CE701205AE71CB50C46694600F0A3
:10E6F00039F8002812D00098019AC10708D0D10734
:10E7000040080843C1435208D0432160606004E0E0
:10E71000D10740080843510803C401201CBDF8B5C7
:10E7200007460020187008700E4610601C461546FB
:10E730006946384600F039F80146012000290AD020
:10E74000009900290CD0C808286000984007400FA5
:10E7500030700120F8BDB968002901D00020F8BD53
:10E760002070FBE7F3B5002681B03446354603E060
:10E77000402E01D30020FEBD6946019800F068F9E3
:10E780000028F8D06846077832467806400EC10F58
:10E79000FDF7D8FA29430443F61D0D463806E7D4A1
:10E7A0000298046041600120FEBDF8B50E460746A0
:10E7B000694600F04DF900280AD068460478200622
:10E7C00016D507256406640E03E0202D01D3002032
:10E7D000F8BD6946384600F03BF90028F8D0684695
:10E7E00001784806400EA8400443ED1D0806ECD40D
:10E7F00001203460F8BD00005968064A89689142DA
:10E8000006D141688068044A491C401E116050606E
:10E8100070470000D8F40300F425002001600023B5
:10E820008360C26041608B789A1803230261CB56E3
:10E83000D21842610878002800D00120704770B5D6
:10E8400045680E46044660680178B14206D14078BA
:10E850000007000F082801D0012070BD204600F0FD
:10E8600005F86068A842EED1002070BD30B541685F
:10E870000A78002A0CD00B460C3343600A7B002A2E
:10E8800008D04C780A79A506AD0F032D07D00BE010
:10E89000002030BDC2680168FFF7C0FFF8E75D786F
:10E8A000AD06AD0F032D06D02509022D09D0A40910
:10E8B000022C09D009E08D7804690022641B0461F0
:10E8C00003E04C79624300E0042249788906890F0D
:10E8D00002D18168491C81609C78016909198918F5
:10E8E000032201619A5689184161012030BD30B57B
:10E8F00041680024497887B00A07120F082A10D00F
:10E900008A091DD08A09022A09D102698906890F5C
:10E910001460022901D0032901D14069047007B0B5
:10E9200030BD0069056808E02C7329466846FEF78B
:10E930004DFB6846FFF7DBFFAD68002DF4D1EEE735
:10E940008906890F012911D00229E6D00329E4D0D4
:10E95000426851780907090F07290AD091680029F0
:10E960000CD012790069FDF7FDF9D8E741690C7008
:10E97000EEE70169906800F02AF8D0E711790069A4
:10E98000FDF709FACBE7000010B5024B002408C0E0
:10E9900016C010BDC3C6030038B50D46044669460F
:10E9A000FFF703FF00280BD0E368A16805CCEB60FC
:10E9B000A96005C50098083C083D814201D20020AD
:10E9C00038BDA860A168081AA060012038BD00B554
:10E9D0000A4687B001466846FFF720FF002807D0A7
:10E9E0006846FFF784FF6846FFF740FF0028F7D12D
:10E9F00007B000BD7FB514460546002915D1134A5E
:10EA00002868904208D110E0102269462846FFF796
:10EA1000F1FF002807D0103C102CF5D8224669469B
:10EA20002846FFF7E7FF04B070BDA868A04201D2F6
:10EA30000020F8E72B682246284698470028F2D0A5
:10EA4000A868001BA8600120EDE70000C3C6030012
:10EA500010B504468068002809D0236801222046AA
:10EA60009847002803D0A068401EA060012010BD78
:10EA700038B50024002907D0012913D0022913D06A
:10EA800005291FD0002038BD0546012269462846C9
:10EA9000FFF7B0FF002813D0684600780006F4D4D2
:10EAA000012038BD08220EE005466946FFF77DFECD
:10EAB000002805D000212846009AFFF79BFF38BDAB
:10EAC000204638BD04220021F7E700000848416EC7
:10EAD000491E416604D10749FD230A781A400A708D
:10EAE000016E491C0166042901D1002101667047AD
:10EAF000443100206426002070B50C490446486E5D
:10EB0000042810D00A6E1218042A00D3121F401CC9
:10EB1000486618204243551801462846FDF73BF940
:10EB20000120256070BD002070BD00004431002030
:10EB300010B518481822016E51430C18406E002879
:10EB40001FD0207A012802D0022816D10FE0A18A16
:10EB5000E08A091AFF2901DC8AB201E0FF220132B2
:10EB6000E168800023690918181829DF01E0A089ED
:10EB700028DF112806D0002803D00921204600F004
:10EB80002FF910BD0449FD220878104004221043DB
:10EB9000087010BD443100206426002010B50548DF
:10EBA00001784A07920F04D1022211430170FFF746
:10EBB000BFFF10BD64260020016806C98A4201D348
:10EBC000501A70478068401A401C80187047F8B58A
:10EBD0001E681C4615460746002904D0012917D097
:10EBE000052921D118E000202060401C2060B0429F
:10EBF0001AD8012229463846FFF7FCFE002806D025
:10EC000028786D1C000601D52068EEE70120F8BDCC
:10EC100008200246186002E00420024618602946D7
:10EC20003846FFF7E7FEF8BD0020F8BDF7B5114DF7
:10EC30000A46064628881049884218D0287AC00714
:10EC400015D00E4C60202070032161700120A0704F
:10EC5000E11C104600F0D2FBC71CE119029800F03D
:10EC6000CDFBC219B189288800F0DEF8FEBD08206E
:10EC7000FEBD000010260020FFFF0000842C0020B5
:10EC8000FFB5144D0A4606462888134981B08842CC
:10EC90001ED0287AC0071BD0104C6020207006219F
:10ECA00061700120A070E11C104600F0A7FBC71C9A
:10ECB000E119039800F0A2FBC719E119049800F0CC
:10ECC0009DFBC219B189288800F0AEF805B0F0BDEF
:10ECD0000820FBE710260020FFFF0000842C002006
:10ECE00070B50A4B04461888094DA8420CD01B7A0F
:10ECF000DB0709D0074B60251D7059709A700322FD
:10ED0000A18900F091F870BD082070BD1026002088
:10ED1000FFFF0000842C002070B501240B49600423
:10ED200008600B4940108860094940398860094DE6
:10ED30006C602F20FEF76CFAAC60074D00242F208A
:10ED4000AC60FEF765FAAC7070BD000080E100E0D9
:10ED500040130140001001403826002010B5044641
:10ED6000FDF734F900280CD0A007C00E002C0ADAF9
:10ED70002107090F08398908144A89008918C969C7
:10ED800006E0134810BDA108124A890089180968D5
:10ED9000C1400806800F042811D200280FD0022895
:10EDA0000DD00D494B68E206D20E01209040002B99
:10EDB00008D0620992008B5803438B5004E004484A
:10EDC000401C10BD05490860002010BD00ED00E0AA
:10EDD0000120000000E400E05C26002000E100E0EB
:10EDE0001FB500220092019202920392037A012B36
:10EDF00002D0022B11D106E06B461A700269029212
:10EE0000828A9A8109E001236A4613708289C38944
:10EE1000D31A6A461381838953814268019200683C
:10EE20008268684690471FBD07B584B000220092F3
:10EE300001926A4611800121917006A9029103494D
:10EE400003916946A6DF07B000BD0000842C0020B6
:10EE5000F8B516460D46040008D0002D06D0206CEB
:10EE6000802200213828225403D307E00E20F8BD69
:10EE70002154401C3828FBD30BE02154401C40286F
:10EE8000FBD32146084600F095F838212046FCF7D0
:10EE900082FF236CA26C590FDB00E06CD218484152
:10EEA0002146A2640306170A2031E0641F43CA7793
:10EEB0008F770304170C1F430302100E4F7718437C
:10EEC0000877E06CC876020A8A76020C4A76000E51
:10EED00008762146084600F06DF8002E1ED000216D
:10EEE000E26EC800C2406A54A36EC3406A18137130
:10EEF000636EC3401372236EC3401373E36DC3404C
:10EF00001374A36DC3401375636DC3401376236DF3
:10EF1000C340491C13770429E2D31FE000211823C2
:10EF2000C800226D181AC2406A54666DC6406A183D
:10EF30001671A66DC6401672E66DC6401673266E33
:10EF4000C6401674666EC6401675A66EC640167626
:10EF5000E66EC640491C16770429E1D30020F8BDAF
:10EF6000002815D0002101648164C164094901654C
:10EF700009494165094981650949C1650949016630
:10EF800009494166094981660949C16600207047FF
:10EF90000E20704767E6096A85AE67BB72F36E3C68
:10EFA0003AF54FA57F520E518C68059BABD9831F54
:10EFB00019CDE05BF0B5CCB0002214460CAB0D19B6
:10EFC0006E782F7836023E43AF7876BA36043F0229
:10EFD000ED783E432E439500521C241D5E51102AAD
:10EFE000EDD320E09100CD18803DAB6F8C4611240D
:10EFF0001946E14113241E46E64171409B0A5940DF
:10F000006B6C07271E46FB4134461227FC415C40CF
:10F01000F3085C4009192C6C6B6E1B19CC18614607
:10F020000CAB5C50521C402ADCD3016D0B91476D38
:10F030000A97836D0993C26D06920092026E089240
:10F04000446E0794A646846E05940194C46E04949D
:10F0500002940024A44606261446F4410B261546C5
:10F06000F5416C4019261546F5416C40019E7546E8
:10F07000154096436E40A6196446A400254D03949E
:10F080002D59029C2C193619039C0CAD2C590D4698
:10F090003419039402260C46F4410D26F5416540CF
:10F0A00016260C46F44165403C465C403E460C400A
:10F0B0001E4074402D19019C029474469646009A95
:10F0C0000194039C00933B460F4612196119644654
:10F0D000641CA446402CBED30B9C611801650A99A0
:10F0E000C91941650999C9188165009B0699C91814
:10F0F000C165089989180166079971444166019AAA
:10F10000059989188166029A04998918C1664CB0DC
:10F11000F0BD000074F60300F0B516460F4604007B
:10F1200005D0002E1ED0002F01D0002518E00E20A3
:10F13000F0BD216C785D6054206C401C2064402838
:10F140000DD121460846FFF735FF0123A16C5B0274
:10F150000022E06CC91822645041A164E0646D1C77
:10F16000B542E6D30020F0BD002803D00249C860B4
:10F17000002070470E207047682600201CB5034908
:10F1800001910091694660DF1CBD0000E025002070
:10F1900070B50E460546144614211046FCF7FBFDDB
:10F1A0000120002120802161217326726572002DCB
:10F1B00000D0A072002070BD10B5002902D0002040
:10F1C000FCF772FFFDF78EFE10BD000010B50021A8
:10F1D000024A0846FCF76AFF10BD0000B9F10300BF
:10F1E00010B5FCF75FFF10BDF8B5002903D08C0700
:10F1F0000025002C01D00720F8BD0E4E0E4FB16047
:10F2000072807360396801246603314203D00A4971
:10F21000254680310E60094910DF002803D0002DFB
:10F22000EAD03E60F8BD034804701620FFF796FD53
:10F23000F8BD00006826002000E100E0E1F10300D5
:10F24000014800787047000068260020002803D09D
:10F2500002490861002070470E2070476826002090
:10F26000FEB51F4C0025A768606802906846FDF750
:10F270000BFD0190FDF7C0FE06460198002822D044
:10F2800000230098616817E00E680A46864202D99A
:10F29000301A086012E0801BF31800261660D6684A
:10F2A000D169B446002E07D0FE183602360A5660E1
:10F2B00066469660D56115460029E5D1284661600D
:10F2C000FDF7F0FE06E02846FDF7ECFE002801D130
:10F2D000002E02D00298FDF713FA0020E070FEBD68
:10F2E0003826002001200249000508607047000010
:10F2F00000E200E010B50E4B5968002906D0026804
:10F300000C68A24204D8A21A0A60C161586010BDFC
:10F310000B4604E00B46C969121B002904D00C6897
:10F320009442F7D3A41A0C600260C161D86110BD89
:10F33000382600207CB50D460646002469460C7030
:10F340006846FCF7F7FF01A800F094F800280DD0FC
:10F35000057046606846084900794870684600783C
:10F36000FDF706F8FFF7BEFF20467CBD6846042483
:10F370000078FCF7FDFFF7E748260020F8B51D4DA3
:10F380006C68002C34D01C4800274068A968401ADB
:10F390000602360A2068B04218D8361AC719224623
:10F3A000107CE46900280FD000201074EB68002B5B
:10F3B00007D0916950699847002805D0FCF774FE82
:10F3C00002E0516990698847002CE3D12978687878
:10F3D000814206D1401CC0B26870022801D10020D1
:10F3E000687004490006800D18310F50FFF77AFF4E
:10F3F000F8BD000038260020001501400870020A00
:10F400004A70020C8A70000EC87004207047000019
:10F4100038B51549154A488890420FD04A78144C9F
:10F42000521CD2B24A70237B934208D3091D75DF68
:10F43000002803D0A169002900D0884738BD0025E5
:10F440004D70217C002907D03B2176DF002803D0B6
:10F45000A169002900D0884761690029EED068467B
:10F460000570884738BD0000FC250020FFFF000024
:10F470000C2C002010B509494B788C785A1CD2B25C
:10F48000944200D100220C78944201D1002010BD9A
:10F490000270486818214B43C01810BD4826002050
:10F4A00010B501E0FDF792FAFDF76CFC0028F9D1E8
:10F4B00010BD00000101000001000000000000007C
:10F4C0000205000021000000000000000000000014
:10F4D0000000000000000000011104FC0400000016
:10F4E00000000000021104FC040000000000000005
:10F4F000032104FC0404000000000000041101FFCB
:10F500000100000000000000051102FE04000000E0
:10F5100000000000061104FC0400000000000000D0
:10F52000071104FC0400000000000000081701FFA0
:10F5300022000000B4F40300091001FF01000000E4
:10F54000B2F4030000000000000000000000000012
:10F5500001010000040000000000000000000000A5
:10F560000000000000000000011101FF0100000088
:10F5700000000000021702FE64000000D8F403003F
:10F58000031704FC0400000050F503000000000015
:10F5900000000000000000000107000070000000F3
:10F5A00068F50300020100000100000000000000F7
:10F5B0000305000041000000000000000000000002
:10F5C0000000000000000000011704FC70000000B3
:10F5D00068F50300021704FCB400000098F503006E
:10F5E00000000000000000000000000015161718C1
:10F5F00011121314EC2B00200010020050EADA3034
:10F600008883B89F604F15F30000C98E0100000089
:10F6100000000000000000000000000001000000E9
:10F6200000000000000000000000000002000000D8
:10F6300000000000000000000000000003000000C7
:10F6400000000000000000000000000004000000B6
:10F6500000000000000000000000000000030000A7
:10F66000383100201431002020000000010000008B
:10F6700000000000982F8A4291443771CFFBC0B53B
:10F68000A5DBB5E95BC25639F111F159A4823F926D
:10F69000D55E1CAB98AA07D8015B8312BE853124C6
:10F6A000C37D0C55745DBE72FEB1DE80A706DC9B87
:10F6B00074F19BC1C1699BE48647BEEFC69DC10F33
:10F6C000CCA10C246F2CE92DAA84744ADCA9B05C6F
:10F6D000DA88F97652513E986DC631A8C82703B032
:10F6E000C77F59BFF30BE0C64791A7D55163CA0640
:10F6F00067292914850AB72738211B2EFC6D2C4D4C
:10F70000130D385354730A65BB0A6A762EC9C28139
:10F71000852C7292A1E8BFA24B661AA8708B4BC2CF
:10F72000A3516CC719E892D1240699D685350EF4F9
:10F7300070A06A1016C1A419086C371E4C774827B0
:10F74000B5BCB034B30C1C394AAAD84E4FCA9C5B26
:10F75000F36F2E68EE828F746F63A5781478C88477
:10F760000802C78CFAFFBE90EB6C50A4F7A3F9BE59
:10F77000F27871C665E403000FE40300B9E3030007
:10F780002BE3030035E30300EDE203003FE3030056
:10F790007BE3030000000000C0F70300E025002029
:10F7A000B0000000AEBF030070F8030090260020F8
:10F7B00060110000BEBF030075C50300F5C403005F
:10F7C0000100000000000000000000000000000038
:10F7D0000000000000000000000000000000000029
:10F7E0000000000000000000000000000000000019
:10F7F000FFFF00000000000000000000000000000B
:10F8000000000000000000000000000000000000F8
:10F8100000000000000000000000000000000000E8
:10F8200000000000000000000000000000000000D8
:10F8300000000000000000000000000000000000C8
:10F8400000000000000000000000000000000000B8
:10F850000000000000000000000000000024F40090
:10F8600000100000000C040045CD03000000000063
:020000041000EA
:0410140000BC030019
:040000050003BCC177
:00000001FF
